:03000000020355A3
:03000B0002015897
:03004300020100B7
:1001000002013C000201180002011800020129004E
:10011000020120000201180032E591C2E4F59122AB
:10012000C0E0C2003119D0E032C0E0E5874401F5FB
:10013000870000003119D0E032C2DC32C0D0C0E00C
:10014000C082C08312016531197401907FABF0D079
:1001500083D082D0E0D0D032C0D0C0E0C082C08393
:050160001203CA80EA51
:10016500907FE8E0A2E79202545C7051E0A2E08241
:10017500E1404A30E50274035403C4F540A3E0545A
:100185000F45401201D12001343002182003209080
:100195007F027846754003E6F0158218D540F8E6EB
:1001A500907FB5F0754002907FB4E04540F0228520
:1001B5008240E583907FD4F0E540A380E675400357
:1001C50080E5E02582F58250020583229001F63113
:1001D500C8E09001F631C8C082C0837845E4F618BE
:1001E500F6187601907FEAE0F5F0A3E0C201C203BC
:1001F500226D404040404081406A7440404040404C
:1002050040714040404040A5404040404040404053
:1002150040714240404040404040404040404040A6
:1002250040405663404040404040435D4040404070
:1002350040D201223000FA907FC5F0907FAAE054A9
:100245000160FBF00203BC3000E70876182230009D
:10025500E0F541223000DA08A64122300004087694
:100265000122760222E5F060061470C5D20022C292
:100275000022D203149002C160B9149002D360B376
:100285001470AE900305E5F0601EF54031C7E060DF
:10029500A0E5401480F2D203C394219002E5609357
:1002A500149002EE608D8089E0FFF5F07800F20889
:0C02B500A3E0DFFAD0E0D0E0E5F021A5E6
:1002C100120101010000004042420001000101024F
:1002D100000109021B000101008032090400000035
:1002E100030000000921000100012217000600FFA0
:1002F1000901A10119012902150026FF00750895C0
:10030100069102C0040309042C0355005300420066
:100311002000440065007300690067006E00200042
:100321004200790020004500780061006D007000F6
:100331006C0065001E034C006900670068007400D2
:1003410069006E0067002000500061006E006500CA
:100351006C0000007581EB75927F78D6E254F3F260
:100361001203ABE24406F2E4F5207893E4F2799CBF
:10037100F4F37895799EE254F0F2E354F0F3758C3E
:1003810050E58954F0D2E1F589E5884430F5887863
:10039100ACF208F2087401F2087401F278AA74FF51
:1003A100F275E80175A8C20080FD75406490FB50AC
:1003B100A3E582458370F9D540F3227847907EC04A
:1003C1007F06E0F6A308DFFA22907F9BE0907F96FC
:1003D100A20430E001B34013A2E09204E4F07847B4
:1003E100794D7F06E6F4F70809DFF9784D7553007A
:1003F1007420C5538640D540024553A64008C553D5
:070401000370EFE553F02248
:00000001FF
